:020000040000FA
:100000003228483461346C346C346F342034A0347A
:100010006F342E346B342E3420342034A0344D34DD
:1000200065347334733465344334A03445346E34EA
:1000300074346C3461346434A0344C3461346434CA
:10004000653420342034A0344B343A3432343034E4
:100050006D344134A0344B343A346D344F34683409
:100060006D34A03483160F178F160F168312860176
:10007000831602308100860103178901031383125E
:10008000860187010715871007158316871007114A
:1000900083128B01312201302322952295229F0168
:1000A0009F1783169F019F170514851403170814C3
:1000B0008814031383121F14071E7620962030081D
:1000C000A3003108A4008821DB212B213808A300DC
:1000D0003908A4008821F921D42088211022083071
:1000E000232295229522952295225C28871E852819
:1000F0002430232207148316071083120714FC20D0
:1001000075218821C42195227F282B3023221F1599
:100110009522FC202308A1002408A20012219F148C
:100120001221FD204E218821F9218828B6200F3088
:100130002322B001B101803083168100831207149D
:100140008316071083120714533081000B11FC2013
:10015000A418B228B00A0319B10A0319B2280B1D5A
:10016000AF28A42883160714831208001630232210
:1001700007108714FC202408031DBA28F830230533
:10018000031DBA28871008001D3023220711FC2008
:10019000FC302404FF3A031DC72807302304FF3A2C
:1001A000031DC72807150800C4202308BA00240827
:1001B000BB009222FC202308A1002408A2003A08D8
:1001C000A3003B08A4004E210318EB28A2012D3008
:1001D000A1005F210800A401A3010800A401A3015C
:1001E000871E08000630A4003730A300B000A1002D
:1001F0003108A2005F2108009F149F18FD281E08E7
:10020000A40083161E088312A30008001F15C8301F
:10021000B500B50B0929FC201F11C830B500B50B7E
:100220000F290800AD01AC0107158714000000007C
:10023000000000000000000000000000871007110F
:1002400000000000000000000000AC0B1429AD0B02
:10025000142907150800EE202308A1002408A20095
:100260001F159522FC2047212308A1002408A20085
:1002700012219F141221FD201F112308B60024080B
:10028000B7004E212308B8002408B900080021084F
:10029000A30722080318220FA4070800261021082C
:1002A000A302031857290130A402031C26142208B4
:1002B000A402031C26140310261803140800B2011C
:1002C000B203B301B303B20A0319B30A4E21031CEC
:1002D00063293208A3003308A4000800A500031016
:1002E000A20CA10CA50B6F2908002308A10024086B
:1002F000A20047214721472147212308A1002408C4
:10030000A20006306E214E2101306E214E210800E0
:100310002730A2001030A100A121A7000330A200C5
:10032000E830A100A121A800A2016430A100A12110
:10033000AA00A2010A30A100A121A9002308AB0054
:100340000800A501A50A4E21031CA2294721250367
:1003500008002308BA002408BB00882189306C22D9
:100360006C22A6142708F2212808F22120307D22D1
:100370002A08F2212908F221A6102B08F2213A08B6
:10038000A3003B08A400080080306C22A6142708B4
:10039000F2212808F22120307D222A08F2212908A2
:1003A000F221A6102B08F22120307D226D307D2213
:1003B00056307D22080080306C22A6142708F221D6
:1003C0002808F22120307D222A08F2212908F22172
:1003D000A6102B08F22120307D22E4307D22463009
:1003E0007D220800031DA6103038A61820307D227B
:1003F0000800C0306C22A6142708F2212808F22138
:1004000020307D222A08F2212908F221A6102B088B
:10041000F22120307D226D307D22F4307D220800D3
:1004200089306C2220307D22A6142A08F221290866
:10043000F221A6102B08F22120307D22E4307D220B
:1004400041307D220800B400CA306C22B4032E2251
:10045000803E03187D2A7F397D22272AB40A34087A
:100460008200952230308600061400000610922289
:1004700030304B2230304B2220304B2201306C2266
:1004800028306C2208306C2206306C2203306C223B
:100490000C306C220800860086110611061400003C
:1004A00006100A30AC00982208008316F03086044B
:1004B000831206118615061400000608AE00061009
:1004C0000000061400000610AE1B592A8611831680
:1004D0000F30860583120800AF00552286110611E1
:1004E0002F08F03986000614000006102F0EF03990
:1004F00086000614000006100800AF0055222F08E1
:10050000F039860006150614000006102F0EF0398B
:100510008600061506140000061006110800643057
:10052000AC00982A3230AC00982AFA30AC00982AF5
:10053000C830AD0000000000000000000000000016
:0C0540000000AD0B9A2AAC0B982A003486
:02400E00E520AB
:02401000FF3F70
:00000001FF
